:100000000C94E7000C9404010C9404010C9404017A
:100010000C9404010C9404010C9404010C9404014C
:100020000C9404010C9404010C9404010C9404013C
:100030000C9404010C9404010C9410070C9404011A
:100040000C9404010C9404010C94C7060C94040154
:100050000C9404010C9404010C9404010C9404010C
:100060000C9404010C9404010C9404010C940401FC
:100070000C9404010C94EB060C9404010C94040100
:100080000C9404010C9404010C9404010A0A0A5310
:100090004552564F20544553542050524F475241D9
:1000A0004D0A0A003E3E3E2000494E56414C49440E
:1000B0000A00082008000A56616C696420436F6DCD
:1000C0006D616E64733A0A0A2020737461747573EB
:1000D000202D207072696E74732063757272656E64
:1000E0007420736572766F2072617720616E642070
:1000F00072656C61746976652D66726F6D2D6365CE
:100100006E7465720A2020202020202020202020CC
:10011000706F736974696F6E730A0A202073657259
:10012000766F203C73313E203C73323E203C73336B
:100130003E203C73343E203C73353E203C73363EBB
:100140000A2020202020202020202D2073657420CC
:10015000616C6C2073697820736572766F7320749C
:100160006F207468652073706563696669656420D3
:10017000706F736974696F6E732E0A2020202020BF
:100180002020202020205A65726F203D2063656E5C
:100190007465722C206D6178203D20313030302C18
:1001A000206D696E203D202D313030300A0A20202C
:1001B0003F202020202020202D2074686973206893
:1001C000656C70206D6573736167650A0A001124A0
:1001D0001FBECFEFD0E1DEBFCDBF11E0A0E0B1E0A8
:1001E000ECE4F1E200E00BBF02C007900D92AA3BE5
:1001F000B107D9F712E0AAEBB1E001C01D92AD350D
:10020000B107E1F70C94490A0C9400002F923F9239
:100210004F925F926F927F928F929F92AF92BF9216
:10022000CF92DF92EF92FF920F931F93CF93DF93C2
:10023000CDB7DEB726970FB6F894DEBF0FBECDBFA1
:100240005C016A017B01522E180127FF02C0552470
:1002500005C085E2821714F485E2582ED5019896E0
:10026000BE83AD8320E030E040E050E0C701B6013E
:100270000E94AE0E882354F4F10180819181826046
:1002800091838083F7FAF094F7F8F094AE014F5F12
:100290005F4FC701B6010E940E0F3B014C01E98080
:1002A000FA800B811C8120E030E040E050E0C80182
:1002B000B7010E94AE0E8823E9F1CD80DE80442490
:1002C00028C02DEC3CEC4CEC5DE3C801B7010E946A
:1002D0003E0FAE014F5F5F4F0E940E0F2AE939E9D2
:1002E00041E251E40E943E0F0E94930E605DD601F0
:1002F0006E936D014394E980FA800B811C8120E0AC
:1003000030E040E050E0C801B7010E94AE0E882303
:1003100019F0AC14BD04A8F2750106C0F601819174
:100320006F01D7018D937D01ED81FE81CE16DF0631
:10033000A8F329C020E030E040E050E0C401B30160
:100340000E94B10E18161CF0750144241CC04424F0
:1003500003C04A943701480120E030E040E251E414
:10036000C401B3010E943E0F7B018C0120E030E00C
:1003700040E85FE30E94AE0E87FDEBCFE982FA8290
:100380000B831C837501D1014D915C9153FF13C008
:10039000BDEF4B1684F0242D332727FD3095852D96
:1003A000992787FD909501962817390724F4546002
:1003B000F10151834083D1018D919C9192FD08C040
:1003C0005394052D112707FD10950A0D1B1D0CC018
:1003D000052D112707FD10950A0D1B1D842D99274A
:1003E00087FD9095080F191F0A151B05D8F4F50114
:1003F0004CC020E030E040E251E4C401B3010E946F
:100400003E0FAE014F5F5F4F0E940E0F3B014C014C
:1004100069817A818B819C810E94930E605DD701F6
:100420006D937D010E151F0528F0ED81FE81EE16FE
:10043000FF06F8F28D819E810817190718F0F50163
:1004400017A224C0D8018C918B5F8C93F80131E303
:1004500018C020E3D8012C93A016B10628F48E9181
:100460008D018F5F8C930DC0D8013C934394D101D3
:100470008D919C9192FF05C0AE16BF0608F42083B3
:100480003196D8018C918A3324F71082842D9927D4
:1004900087FD909526960FB6F894DEBF0FBECDBFB0
:1004A000DF91CF911F910F91FF90EF90DF90CF9050
:1004B000BF90AF909F908F907F906F905F904F9084
:1004C0003F902F9008952F923F924F925F926F929C
:1004D0007F928F929F92AF92BF92CF92DF92EF92D4
:1004E000FF920F931F93CF93DF93CDB7DEB7EE97B5
:1004F0000FB6F894DEBF0FBECDBFCC24DD2476014D
:100500003C017EAF6DAF5A011A821982FC0117823D
:100510001682838181FDF3C38FEF9FEF16C409819B
:100520001A8100FFD3C3842D80538A30D0F4F0E3C6
:100530004F1631F4552021F403FD02C0116075C13E
:100540008AE0252D2802C0011124542C580E30EDCC
:10055000530E57FE02C04FE7542E03FDCAC3352C7D
:10056000C8C3442D45564CAF433028F0842D8554E4
:10057000833008F0FCC0C501049698AF8FABF5013D
:10058000C080D180E280F38003FD02C036E0532EAC
:10059000077B1A83098346015701A7019601C7010A
:1005A000B6010E94790A8823C1F08EE48D838B8383
:1005B00081E48C839E012A5F3F4F3AAF29AF3CAD67
:1005C000333008F07AC28B81805E8B838C81805EB1
:1005D0008C838D81805E8D8370C2C701B6010E94BD
:1005E000050F892BE9F089E48D838EE48C8386E402
:1005F0008B8320E030E040E050E0C701B6010E946C
:10060000AE0E87FD06C0AE014A5F5F4F5AAF49AFDD
:10061000D6CF8DE28E83CE0107969AAF89AFCFCF2A
:10062000C80192609A838983E7E44E1609F449C0B1
:10063000E41544F0F5E44F1679F026E4421609F08B
:1006400042C31DC036E64316D1F047E64416C9F151
:1006500055E6451609F037C38E010F5F1F4F252D54
:10066000B501A401CE010F960E940601282E8CEF41
:10067000380E15140CF43A94DE011F9615C09460E0
:100680009A8389838E010F5F1F4F252DB501A40129
:10069000CE010F960E940601282E15140CF43A94F0
:1006A000DE011F96121444F4FD0101900020E9F7C9
:1006B0003197CE2ECA1A02C0C52CC394BAAFA9AFC7
:1006C0007DC1552011F0252D01C021E098609A834D
:1006D00089838E010F5F1F4FB501A401CE010F96D4
:1006E0000E940601282E89819A8192FF1EC0822DC8
:1006F000850D8150282FA82FBB27A7FDB095AC0FE3
:10070000BD1F1F9605C08C9111972150803331F485
:10071000622F27FD23C02215B4F703C3C62E562E21
:100720005218539400C3C92E17C0252DE52DFF275D
:10073000E7FDF095EC0FFD1F3F9606C080813197D5
:10074000292F2150803379F7922F1216BCF3522EA5
:10075000C22E222309F4EFC2592EEDC2E22FFF2749
:10076000E7FDF095EC0FFD1F108A552499CFC801C5
:100770008870907003FF04C0552011F421E0522EC0
:10078000E9E64E1609F493C0E4153CF1F3E54F1683
:1007900009F474C0F415ACF02BE24216E1F1241513
:1007A00044F030E24316D1F143E2441609F080C22E
:1007B0003FC05DE24516C1F18EE2481609F078C2ED
:1007C00039C093E64916E1F1E4E64E1609F46FC02C
:1007D000F8E54F1609F06CC29FC020E7421609F4F5
:1007E00096C0241544F03CE6431641F14FE644160A
:1007F00009F05EC20DC055E7451609F48FC0E8E761
:100800004E1609F489C0F3E74F1609F051C221C012
:1008100028E02BAF83C000611A83098389819A8104
:1008200080629A83898365C200681A83098361C2E2
:100830000064FBCF08601A83098352C20460F5CFBD
:10084000A5014E5F5F4F58AF4FABF501C0803A94A2
:1008500034C1F501C080D180892B41F0652D772707
:1008600067FD7095C6010E94A00C18C0F6010190AA
:100870000020E9F73197EC19EBAF11C0F501C0800A
:10088000D180892B41F0652D772767FD7095C601D2
:100890000E948B0C03C0C6010E94820C8BAF950195
:1008A0002E5F3F4F38AF2FAB3BAD331A06C102FF6F
:1008B0000BC0A5014C5F5F4F58AF4FABF501608196
:1008C0007181828193810EC095012E5F3F4F38AFB9
:1008D0002FABF501808191819C01B901882777FDBB
:1008E0008095982F6B017C0197FF0BC002601A83E3
:1008F0000983F094E094D094C094C11CD11CE11CF5
:10090000F11C89819A818F7B9A83898327C0006437
:100910001A83098398E7492E30E13BAF29813A8158
:1009200022FF0BC0A5014C5F5F4F58AF4FABF501E5
:1009300060817181828193810CC0A5014E5F5F4F00
:1009400058AF4FABF50180819181AC01BA01882786
:1009500099276B017C012F7C3A83298387017601DB
:10096000CE0103969AAF89AF9BADA92EBB24CC24B0
:10097000DD24C801B701A60195010E9408106A3064
:100980001CF0640D615201C0605DE9ADFAAD619388
:10099000FAAFE9AFC801B701A60195010E9408109E
:1009A00079018A01211531054105510511F7CC2442
:1009B000DD247601CE010396C9ACC81A49815A815B
:1009C000CA0182739070892B09F03A9446FF07C0E0
:1009D000FBADF03111F482E001C081E0381A43FF31
:1009E00010C0252D332727FD30958C2D9927821790
:1009F000930724F0477F5A83498303C05C18351856
:100A000001C03C1840785170452B69F4832D06C015
:100A1000B30180E290E00E94FB0C812F182F11504F
:100A20001816B4F3312E89819A8181FF04C0B30175
:100A30008DE290E00BC084FF04C0B3018BE290E034
:100A400005C085FF05C0B30180E290E00E94FB0C69
:100A500089819A8186FF0FC0B30180E390E00E94F4
:100A6000FB0C2BAD203139F4B301842D992787FD80
:100A700090950E94FB0C89819A8190FF0DC0832D77
:100A800006C0B30180E390E00E94FB0C812F182F79
:100A900011501816B4F3312E89819A8183FF0DC04D
:100AA000252D06C0B30180E390E00E94FB0C212FAE
:100AB000122F11501216B4F3512E898187FD0DC0EB
:100AC000832D06C0B30180E290E00E94FB0C812FD1
:100AD000182F11501816B4F3312E33E6431631F4A3
:100AE000B3018C2D992787FD9095BEC043E744162E
:100AF000B1F4460156011BAD09C0F50181915F01BA
:100B0000B301992787FD90950E94FB0C1150A8F71F
:100B10006401FBADCF0ED11C2FEF2BAFB8C033E576
:100B20004316B1F446018601BBAC08C0F8018491BC
:100B3000B30199270E94FB0C0F5F1F4FBA94FFEF80
:100B4000BF16A1F764012BADC20ED11CFBAF9FC035
:100B500089819A8191FD03C009AD1AAD91C092FFC0
:100B60001DC01214BCF4A9ACBAAC122D09C0F50119
:100B700081915F01B301992787FD90950E94FB0C3D
:100B80001150A8F729AD3AAD220D311D3AAF29AF6A
:100B900022240FC0B30180E390E009C0E9ADFAADB3
:100BA0008191FAAFE9AFB301992787FD90950E9433
:100BB000FB0C15142CF4B3018EE290E00E94FB0CA8
:100BC00089819A8192FD06C017C0B30180E390E04D
:100BD0000E94FB0C2394822D815087FF0DC05A94F4
:100BE000852D8F5F18168CF307C0B301892F9927C5
:100BF00087FD90950E94FB0CE9ADFAAD9191FAAF9B
:100C0000E9AF992329F05A94852D8F5F18166CF35C
:100C100089819A8192FD3BC0B301842D992787FD7C
:100C200090950E94FB0C2A9427FE07C0B3018DE229
:100C300090E00E94FB0C219405C0B3018BE290E090
:100C40000E94FB0C6AE070E0822D992787FD909549
:100C50000E94F50F6B017C01CB01C096B3010E948D
:100C6000FB0CB301C701C0960E94FB0C10C0F80139
:100C700082918F01B301992787FD90950E94FB0C0B
:100C8000CE0103960817190791F71AAF09AF8981AA
:100C900087FF17C0832D06C0B30180E290E00E9459
:100CA000FB0C812F182F11501816B4F3312E09C0E8
:100CB000B301842D992787FD90950E94FB0CB8AE57
:100CC000AFAA1A821982AFA8B8AC13C0F5E24F16CA
:100CD00049F481E090E09A8389832AE02BAF3324A2
:100CE000552407C0B301842D992787FD90950E9454
:100CF000FB0C4DAD5EAD4F5F5F4F5EAF4DAFF3018F
:100D0000838183FF04C0EDADFEAD449003C0EDAD23
:100D1000FEAD4080442009F002CCF301868197812A
:100D200014C0C22E5524EC2DFF27E7FDF095EC0FE3
:100D3000FD1F108AB2CCEC2DFF27E7FDF095EC0FDC
:100D4000FD1F108AFEEF4F0E92CCEE960FB6F89470
:100D5000DEBF0FBECDBFDF91CF911F910F91FF90EE
:100D6000EF90DF90CF90BF90AF909F908F907F904B
:100D70006F905F904F903F902F9008955D9BFECFB6
:100D80008CB980E090E008950E94BE0608951F92FD
:100D90000F920FB60F9211248F93CF93DF93CDB79D
:100DA000DEB72197DEBFCDBF8BB189838CB1809335
:100DB0005002898184FD03C081E080934F02219617
:100DC000F894DEBFCDBFDF91CF918F910F900FBE12
:100DD0000F901F9018951F920F920FB60F9211242B
:100DE0008F93AF93BF93EF93FF931092890010926C
:100DF0008800EBE8F0E080818C6F8083ACE8B0E0A5
:100E00008C91806E8C9380818B7A8083FF91EF919F
:100E1000BF91AF918F910F900FBE0F901F901895BB
:100E20001F920F920FB60F9211248F93EF93FF939F
:100E30001DBC1CBC8FB58C6F8FBDEAE7F0E08081D4
:100E4000806E80838FB58B7A8FBDFF91EF918F91EC
:100E50000F900FBE0F901F901895EF92FF920F9377
:100E60001F93F701ACEF88319A071CF480ED97E0EF
:100E700009C0A3E0893E9A071CF080EA9FE002C007
:100E80008854944F90938700809386008CEF68314C
:100E900078071CF460ED77E009C0A3E0693E7A07AB
:100EA0001CF060EA7FE002C06854744F70938500C4
:100EB000609384008CEF483158071CF440ED57E0F4
:100EC00009C0A3E0493E5A071CF040EA5FE002C0B7
:100ED0004854544F50938300409382008CEF283144
:100EE00038071CF420ED37E009C0A3E0293E3A079B
:100EF0001CF020EA3FE002C02854344F3BBD2ABD1D
:100F00008CEF083118071CF400ED17E009C0A3E0CE
:100F1000093E1A071CF000EA1FE002C00854144FF3
:100F200019BD08BD8CEFE831F8071CF480ED97E09F
:100F30000AC0A3E0E93EFA071CF080EA9FE003C084
:100F4000CF018854944F90937900809378001F913B
:100F50000F91FF90EF90089582B1886382B9EBE81A
:100F6000F0E0808184758083808184658083EAE8F5
:100F7000F0E08081827E8083808182608083109215
:100F8000890010928800ECE8F0E08081806E808318
:100F9000EDE7F0E080818460808387B3806E87BB5B
:100FA0008FB584758FBD8FB584658FBD8EB5827EFC
:100FB0008EBD8EB582608EBD1DBC1CBCEAE7F0E024
:100FC0008081806E808387B7846087BF88EB9BE0D9
:100FD000909387008093860090938500809384008F
:100FE00090938300809382009BBD8ABD99BD88BD8C
:100FF00090937900809378000895CF92DF92EF92DA
:10100000FF920F931F93CF93DF93CDB7DEB7229755
:101010000FB6F894DEBF0FBECDBF8C016B017A0115
:1010200040E050E0BE016F5F7F4F0E94480BE981B6
:10103000FA810E171F0721F080818032E1F021C074
:101040001F930F9380E091E09F938F930E94280D50
:10105000D6010D931C930F900F900F900F90E114F9
:10106000F10419F46FEF7FEF14C081E0F701808382
:101070006FEF7FEF0EC03196FA83E9838081803273
:10108000D1F3D601ED93FC93E114F10411F0F701D3
:101090001082CB0122960FB6F894DEBF0FBECDBFF3
:1010A000DF91CF911F910F91FF90EF90DF90CF9044
:1010B00008952F923F924F925F926F927F928F92FC
:1010C0009F92AF92BF92CF92DF92EF92FF920F93D7
:1010D0001F93CF93DF93CDB7DEB725970FB6F89464
:1010E000DEBF0FBECDBF182F8D3019F08A3009F04A
:1010F0006EC18AE00E94BE068091BA01EBEBF1E07E
:10110000E80FF11D10828091BB01882309F454C1BE
:10111000E090B201F090B301F701108220E030E0DE
:101120006BEB71E00AC0F701E40FF51F8C9180832F
:101130002F5F3F4F2431310509F1A901D901A60FD5
:10114000B71F8C91882311F0803269F7F701E20F05
:10115000F31F1082890105541E4FF80180818032EF
:1011600031F40F5F1F4FF80180818032D1F3F80115
:101170008081882339F400E010E004C0F701138A6D
:1011800000E010E0F7018081882309F415C168E2CE
:1011900071E0C7010E94960C892B49F486EB90E020
:1011A0009F938F930E94480D0F900F9005C16AE2A4
:1011B00071E0C7010E94960C892B09F071C0E6E826
:1011C000F0E08081918120813181885B9B409F93F9
:1011D0008F933F932F9381E391E09F938F930E948E
:1011E000280DE4E8F0E08081918120813181885BE5
:1011F0009B409F938F933F932F9383E491E09F9322
:101200008F930E94280DE2E8F0E080819181208197
:101210003181885B9B409F938F933F932F9385E50C
:1012200091E09F938F930E94280D8AB59BB52AB5B4
:101230003BB5885B9B409F938F933F932F9387E6AB
:1012400091E09F938F930E94280D88B599B528B59A
:1012500039B5885B9B409F938F933F932F9389E78A
:1012600091E09F938F930E94280DE8E7F0E0808142
:10127000918120813181885B9B409F938F933F9325
:101280002F938BE891E09F938F930E94280D8DB749
:101290009EB784960FB6F8949EBF0FBE8DBF8CC0CC
:1012A0006DE971E0C7010E94960C892B09F074C0AA
:1012B0000115110509F480C01B830A83CC24DD24A9
:1012C0006894C1F8CC0EDD1E5E010894A11CB11C0F
:1012D000A501B601C8010E94FD073C019F938F93B1
:1012E00083EA91E09F938F930E94280DE980FF2469
:1012F000E7FCF094A501B6018A819B810E94FD075D
:101300009D838C838981992787FD9095E80EF91E2E
:10131000A501B6018A819B810E94FD072C010981EC
:10132000112707FD1095A501B6018A819B810E94B6
:10133000FD071C018981992787FD9095080F191FCA
:10134000A501B6018A819B810E94FD074C0189811C
:10135000992787FD9095E80EF91EA501B6018A81AF
:101360009B810E94FD079C018981992787FD9095AB
:10137000080F191FE00EF11E0F900F900F900F90A5
:10138000EF28D1F4790184019101A2016C817D8162
:10139000C3010E942D0710C089EA90E09F938F93AC
:1013A0000E94480D86EB90E09F938F930E94480D1A
:1013B0000F900F900F900F9084EA90E09F938F937F
:1013C0000E94480D1092BA010F900F9049C08830CA
:1013D000D9F48091BA018823D1F182EB90E09F93F8
:1013E0008F930E94480D8091BA010F900F9088232F
:1013F00019F081508093BA018091BA01EBEBF1E0D2
:10140000E80FF11D10822CC00E94BE068091BA0127
:10141000EBEBF1E0E80FF11D10838F5F8093BA01D1
:101420008038F1F41092BA011092BB0189EA90E081
:101430009F938F930E94480D84EA90E09F938F932F
:101440000E94480D0F900F900F900F9009C088E0F8
:101450000E94BE0688E08093BB0181E08093BA01C0
:1014600025960FB6F894DEBF0FBECDBFDF91CF91AA
:101470001F910F91FF90EF90DF90CF90BF90AF90B2
:101480009F908F907F906F905F904F903F902F90A4
:101490000895CFEFD0E1DEBFCDBF1092900087E678
:1014A00089B988E98AB90E94AC07789460E070E055
:1014B00084EC96E00E94AB0C8CE890E09F938F93B5
:1014C0000E94480D84EA90E09F938F930E94480DFC
:1014D0000F900F900F900F9080914F028823E1F3AF
:1014E000F89410924F028091500278940E9459080B
:1014F000F3CFA8E1B0E0EFE7FAE00C944E10698377
:101500007A838B839C832D833E834F835887BE01D0
:10151000675F7F4FCE0101960E94A90ABE016F5EF0
:101520007F4FCE0105960E94A90A8985823018F462
:1015300081E090E00AC020E030E08989823010F03C
:10154000C90103C021E030E0C901E2E068960C94D3
:101550006A10FC01DB01208131819281492F4F7794
:1015600050E0991F9927991F8381682F660F692B77
:10157000881F8827881FFD018183662309F049C0E1
:10158000211531054105510509F470C082E89FEF2E
:10159000FD0193838283220F331F441F551F220FA7
:1015A000331F441F551F220F331F441F551F220F87
:1015B000331F441F551F220F331F441F551F220F77
:1015C000331F441F551F220F331F441F551F83E035
:1015D0008C932030F0E03F07F0E04F07F0E45F0726
:1015E00090F482E89FEF220F331F441F551F01978D
:1015F000203060E0360760E0460760E4560798F365
:10160000FD0193838283FD012483358346835783C1
:1016100008956F3F71F1862F99278F579040FD01F4
:101620009383828383E08C93220F331F441F551FC3
:10163000220F331F441F551F220F331F441F551FF6
:10164000220F331F441F551F220F331F441F551FE6
:10165000220F331F441F551F220F331F441F551FD6
:1016600050642483358346835783089582E08C93A6
:101670000895211531054105510519F484E08C9335
:10168000089544FD02C01C92BECF81E08C93BBCF75
:101690002F923F924F925F926F927F928F929F9282
:1016A000AF92BF92CF92DF92EF92FF920F931F9370
:1016B000CF93DF93CDB7DEB723970FB6F894DEBF95
:1016C0000FBECDBF9B838A831B016A016115710523
:1016D00019F0FB0191838083C114D10449F0C60144
:1016E0000297839728F040E050E060E070E0EFC0A0
:1016F000EA81FB811191FB83EA83812F99270E9464
:101700007510892BA9F71D3241F4EA81FB811191F3
:10171000FB83EA83F1E0F98308C01B3229F4EA81F4
:10172000FB811191FB83EA831982C114D10421F05A
:10173000F0E1CF16D10439F51033A1F4EA81FB8131
:101740008081883711F0883569F4EA81FB81118145
:101750003296FB83EA83F981F260F98360E1C62E59
:10176000D12C11C0C114D10471F4103359F55FEFBD
:10177000852E5FEF952E5FEFA52E5FE1B52E48E039
:10178000C42ED12C38C08AE0C816D104F1F090E103
:10179000C916D10429F0E8E0CE16D104F9F409C045
:1017A0003FEF832E3FEF932E3FEFA32E3FE0B32E6C
:1017B00022C02FEF822E2FEF922E2FEFA22E2FE19D
:1017C000B22E19C09AE0C92ED12C89E9882E89E958
:1017D000982E89E9A82E89E1B82E0DC096014427DC
:1017E00037FD4095542F6FEF7FEF8FEF9FEF0E94F3
:1017F000081049015A0140E050E060E070E030E03C
:101800002601662457FC6094762C212F20532A3021
:1018100060F0812F81548A3110F4275006C0812F47
:1018200081568A3160F5212F2755822F99278C15F3
:101830009D052CF537FD1DC084169506A606B70636
:10184000B8F0E22EFF2400271127CB01BA01A30133
:1018500092010E948710AB01BC014E0D5F1D601FFD
:10186000711F4E155F056007710710F031E001C070
:101870003FEFEA81FB811191FB83EA83C6CF2114FC
:10188000310479F0332321F08A819B81019706C0CE
:10189000F981F1FF06C08A819B810297F101918352
:1018A0008083F981F0FF07C0709560955095419550
:1018B0005F4F6F4F7F4F37FF0AC082E290E09093F7
:1018C0005802809357024FEF5FEF6FEF7FEFCB012E
:1018D000BA0123960FB6F894DEBF0FBECDBFDF91DD
:1018E000CF911F910F91FF90EF90DF90CF90BF901D
:1018F000AF909F908F907F906F905F904F903F90B0
:101900002F900895FC0105900020E9F780959095AF
:101910008E0F9F1F0895FC010590615070400110CB
:10192000D8F7809590958E0F9F1F0895FB01DC01DD
:101930008D910190801911F40020D1F7990B089531
:10194000FC016150704001900110D8F7809590958E
:101950008E0F9F1F0895EF92FF920F931F93CF93C7
:10196000DF938C017B01892B11F4672BD1F16EE0A1
:1019700070E081E090E00E94770DFC01009789F112
:10198000DC0180E88383E114F10471F0F386E286E0
:1019900081E883838091510290915202892B21F436
:1019A000F0935202E093510201151105E1F0118705
:1019B00000878381826083838091530290915402D7
:1019C000892B89F4F0935402E093530280915502DD
:1019D00090915602892B39F4F0935602E093550208
:1019E00002C0A0E0B0E0CD01DF91CF911F910F9137
:1019F000FF90EF9008950F931F93CF93DF938C0187
:101A0000EB018B81992781FF1BC082FF0DC02E81C6
:101A10003F818C819D812817390764F4E881F98121
:101A20000193F983E88306C0E885F985802F09953D
:101A3000892B31F48E819F8101969F838E8302C012
:101A40000FEF1FEFC801DF91CF911F910F91089504
:101A5000CF93DF93CDB7DEB722970FB6F894DEBFF2
:101A60000FBECDBFFE01379661917191FA83E98374
:101A7000AF0180915302909154020E94630222961A
:101A80000FB6F894DEBF0FBECDBFDF91CF910895A2
:101A9000CF93DF93CDB7DEB722970FB6F894DEBFB2
:101AA0000FBECDBFFE01379661917191FA83E98334
:101AB000E0915302F09154028381886083834981CD
:101AC0005A8180915302909154020E946302E091E6
:101AD0005302F09154022381277F238322960FB66D
:101AE000F894DEBF0FBECDBFDF91CF9108950F9365
:101AF0001F93CF93DF93869F8001879F100D969F42
:101B0000100D1124C8010E94930DEC01009729F0DB
:101B1000A80160E070E00E948C0ECE01DF91CF91B1
:101B20001F910F910895CF93DF93AC01029710F4AA
:101B300042E050E0A0915B02B0915C02FD01C0E088
:101B4000D0E020E030E020C08081918184179507AB
:101B500069F482819381209719F09B838A8304C062
:101B600090935C0280935B02CF0132C04817590703
:101B700038F42115310519F08217930708F49C01F8
:101B8000EF010280F381E02D3097F1F62115310548
:101B900089F1C901841B950B049708F4A901E0E0C1
:101BA000F0E026C08D919C91119782179307E9F47C
:101BB0004817590779F4ED018A819B81309719F014
:101BC0009383828304C090935C0280935B02CD0177
:101BD000029649C0841B950BFD01E80FF91F419344
:101BE000519302978D939C933AC0FD01A281B381DA
:101BF0001097C1F68091590290915A02892B41F4B5
:101C00008091B6019091B70190935A028093590246
:101C10002091B8013091B9012115310541F42DB75A
:101C20003EB78091B4019091B501281B390BE0912A
:101C30005902F0915A022E1B3F0B2417350788F0EA
:101C4000CA0102962817390760F0CF01840F951F4B
:101C5000029690935A028093590241935193CF0177
:101C600002C080E090E0DF91CF910895CF93DF93A1
:101C7000009709F44EC0EC0122971B821A82A091B2
:101C80005B02B0915C02109711F140E050E001C09E
:101C9000DC01AC17BD0700F1BB83AA83FE012191D3
:101CA0003191E20FF31FEA17FB0771F42E5F3F4FEC
:101CB0008D919C911197820F931F99838883FD01C9
:101CC000828193819B838A834115510559F4D09376
:101CD0005C02C0935B021DC0FD0182819381AD0156
:101CE0000097B1F6FA01D383C28321913191E20FBB
:101CF000F31FEC17FD0769F42E5F3F4F8881998130
:101D0000820F931FFA01918380838A819B81938341
:101D10008283DF91CF910895DC0101C06D93415022
:101D20005040E0F7089597FB47D09F3738F0FEE921
:101D3000F91B982F872F762F6B2F05C05AC09695C9
:101D4000879577956795F150D0F73EF490958095FB
:101D5000709561957F4F8F4F9F4F08950ED05EF025
:101D600004C00BD026F001C008D019F020F48FEF8A
:101D7000089580E0089581E0089597FB092E0526D7
:101D800000F8689410D0E89407FC07C06217730746
:101D90008407950721F008F4009407949894089517
:101DA000052E092607FA440F551F5F3F79F0AA2731
:101DB000A51708F051E04795880F991F9F3F31F014
:101DC000BB27B91708F091E0879508959F919F91DF
:101DD000112408C197FB880F991F9F3F31F0BB2743
:101DE000B91708F091E0879508959F919F9111246C
:101DF000F9C0662777278827992708959F3F59F4C8
:101E0000803C49F481E099270895906889238723CD
:101E100086238395B9F3882799270895DBDFCF932D
:101E2000DF93D52FC42F5527442733272227992303
:101E3000D9F09F37C8F0F92FBDD0592F482F372F31
:101E4000262FF63968F46FDFA6D0C030CD0721F019
:101E500069937993899399939058DF91CF9157C063
:101E60009927882777276627C030CD0721F0299347
:101E7000399349935993DF91CF919CC091DF01D061
:101E800099C0992339F0552329F09F575F57950F33
:101E900013F49AF1B1CF91589F3FE1F3629FA12DC6
:101EA0000F92BB27639FA00DB11DEE27729FA00D5F
:101EB000B11DEE1FAF93AA27649FB00DE11D739F64
:101EC000B00DE11DAA1F6627829FB00DE11DA61F60
:101ED0005527749FE00DA11D551F839FE00DA11D87
:101EE000561F849FA00D511D852F7A2F6E2F1F9096
:101EF0000F9088231AF4939539F474C0000C111CC8
:101F0000BB1F661F771F881F012808955058192E80
:101F100047DF01D04FC0BA176207730784079507E0
:101F2000B1F188F40EF410940B2EBA2FA02D062ECA
:101F3000622F202D072E732F302D082E842F402D39
:101F4000092E952F502DFF275523B9F0591B49F025
:101F5000573E98F0469537952795A795F0405395AD
:101F6000C9F776F0BA0F621F731F841F30F487958C
:101F700077956795B795F040939517FA0F2E0895CA
:101F8000BF1BBB27BA0B620B730B840BF6CFDEF6BD
:101F900033CFE89403C097FB0EF4D8DEB62F672F3B
:101FA000782F892F9EE9002405C09A95BB0F661FE4
:101FB000771F881F11249923A1F08823B2F79F3F30
:101FC00059F0BB0F48F421F4002011F460FF04C065
:101FD0006F5F7F4F8F4F9F4F881F9795879597F91A
:101FE000089507CF9FEF80EC089597FB092E0726F1
:101FF0000AD077FD04D02ED006D000201AF47095B8
:1020000061957F4F0895F6F7909581959F4F0895BC
:10201000A1E21A2EAA1BBB1BFD010DC0AA1FBB1FEC
:10202000EE1FFF1FA217B307E407F50720F0A21B5E
:10203000B30BE40BF50B661F771F881F991F1A94CB
:1020400069F760957095809590959B01AC01BD01F5
:10205000CF010895AA1BBB1B51E107C0AA1FBB1FDC
:10206000A617B70710F0A61BB70B881F991F5A9524
:10207000A9F780959095BC01CD0108952F923F92CC
:102080004F925F926F927F928F929F92AF92BF9288
:10209000CF92DF92EF92FF920F931F93CF93DF9334
:1020A000CDB7DEB7CA1BDB0B0FB6F894DEBF0FBE91
:1020B000CDBF09942A88398848885F846E847D84DE
:1020C0008C849B84AA84B984C884DF80EE80FD80E0
:1020D0000C811B81AA81B981CE0FD11D0FB6F89456
:1020E000DEBF0FBECDBFED01089591110DC080324E
:1020F00051F08A3041F08C3031F08D3021F0893050
:1021000011F08B3099F70895992788270895629FD9
:10211000D001739FF001829FE00DF11D649FE00DDF
:10212000F11D929FF00D839FF00D749FF00D659F40
:10213000F00D9927729FB00DE11DF91F639FB00D3F
:0C214000E11DF91FBD01CF01112408951D
:10214C006572726F723A206765745F6E756D2829BF
:10215C003A2063616E2774207363616E206172672D
:10216C003A20222573220A003F0073746174757340
:10217C0000534552564F31203D20257520282564AB
:10218C00290A00534552564F32203D2025752028F0
:10219C002564290A00534552564F33203D2025759E
:1021AC0020282564290A00534552564F34203D20DF
:1021BC00257520282564290A00534552564F352091
:1021CC003D20257520282564290A00534552564F79
:1021DC0036203D20257520282564290A0073657258
:1021EC00766F0073657474696E6720746F20257543
:0A21FC000A003B0220005D02000013
:00000001FF
